BL51 BANKED LINKER/LOCATER V6.22                                                        11/20/2017  11:41:54  PAGE 1


BL51 BANKED LINKER/LOCATER V6.22, INVOKED BY:
C:\KEIL4\C51\BIN\BL51.EXE .\OBJ\MAIN.obj, .\OBJ\Func.obj, .\OBJ\MCU.obj, .\OBJ\TWI.obj TO .\OBJ\5D_TWI0_M_P22P24_INT PRI
>> NT (.\LST\5D_TWI0_M_P22P24_INT.m51) RAMSIZE (256)


MEMORY MODEL: SMALL


INPUT MODULES INCLUDED:
  .\OBJ\MAIN.obj (MAIN)
  .\OBJ\Func.obj (FUNC)
  .\OBJ\MCU.obj (MCU)
  .\OBJ\TWI.obj (TWI)
  C:\KEIL4\C51\LIB\C51S.LIB (?C_STARTUP)
  C:\KEIL4\C51\LIB\C51S.LIB (?C?CLDPTR)
  C:\KEIL4\C51\LIB\C51S.LIB (?C?CSTPTR)
  C:\KEIL4\C51\LIB\C51S.LIB (?C?CCASE)


LINK MAP OF MODULE:  .\OBJ\5D_TWI0_M_P22P24_INT (MAIN)


            TYPE    BASE      LENGTH    RELOCATION   SEGMENT NAME
            -----------------------------------------------------

            * * * * * * *   D A T A   M E M O R Y   * * * * * * *
            REG     0000H     0008H     ABSOLUTE     "REG BANK 0"
            DATA    0008H     0009H     UNIT         ?DT?TWI
            DATA    0011H     0007H     UNIT         ?DT?_BUFCMP?FUNC
            DATA    0018H     0007H     UNIT         ?DT?_BUFCPY?FUNC
                    001FH     0001H                  *** GAP ***
            BIT     0020H.0   0000H.1   UNIT         ?BI?FUNC
            BIT     0020H.1   0000H.1   UNIT         _BIT_GROUP_
                    0020H.2   0000H.6                *** GAP ***
            DATA    0021H     0002H     UNIT         ?DT?MAIN
            DATA    0023H     0002H     UNIT         ?DT?FUNC
            IDATA   0025H     0004H     UNIT         ?ID?MCU
            IDATA   0029H     0001H     UNIT         ?STACK

            * * * * * * *  X D A T A   M E M O R Y  * * * * * * *
            XDATA   0000H     00C8H     UNIT         ?XD?FUNC

            * * * * * * *   C O D E   M E M O R Y   * * * * * * *
            CODE    0000H     0003H     ABSOLUTE     
            CODE    0003H     0007H     UNIT         ?CO?TWI
                    000AH     0001H                  *** GAP ***
            CODE    000BH     0003H     ABSOLUTE     
            CODE    000EH     0013H     UNIT         ?PR?_TESTOUTSTR?FUNC
                    0021H     0002H                  *** GAP ***
            CODE    0023H     0003H     ABSOLUTE     
            CODE    0026H     003DH     UNIT         ?PR?_TESTOUTBYTE?FUNC
            CODE    0063H     0003H     ABSOLUTE     
            CODE    0066H     00A2H     UNIT         ?PR?TWI0_ISR?TWI
            CODE    0108H     007AH     UNIT         ?PR?TWI0PROC?TWI
            CODE    0182H     0051H     UNIT         ?C?LIB_CODE
            CODE    01D3H     0047H     UNIT         ?PR?MAIN?MAIN
            CODE    021AH     0047H     UNIT         ?PR?INT_UART?FUNC
            CODE    0261H     003DH     UNIT         ?PR?_BUFCMP?FUNC
BL51 BANKED LINKER/LOCATER V6.22                                                      11/20/2017  11:41:54  PAGE 2


            CODE    029EH     0036H     UNIT         ?PR?_BUFCPY?FUNC
            CODE    02D4H     0033H     UNIT         ?PR?_TESTOUTOCT?FUNC
            CODE    0307H     002CH     UNIT         ?PR?_TESTOUTHEX?FUNC
            CODE    0333H     002AH     UNIT         ?PR?_WRITEP?MCU
            CODE    035DH     0027H     UNIT         ?PR?INITSYSTEM?MCU
            CODE    0384H     0025H     UNIT         ?PR?INT_T0?MCU
            CODE    03A9H     001DH     UNIT         ?PR?CHECKTRAPFLAG?MCU
            CODE    03C6H     0016H     UNIT         ?PR?INITUART0?MCU
            CODE    03DCH     0016H     UNIT         ?PR?INITCLOCK?MCU
            CODE    03F2H     0013H     UNIT         ?PR?_NUMBERCHK?FUNC
            CODE    0405H     000FH     UNIT         ?PR?INITPORT?MCU
            CODE    0414H     000CH     UNIT         ?PR?INITTIMER?MCU
            CODE    0420H     000CH     UNIT         ?C_C51STARTUP
            CODE    042CH     000AH     UNIT         ?CO?MAIN
            CODE    0436H     000AH     UNIT         ?PR?INITTWI0?MCU
            CODE    0440H     000AH     UNIT         ?PR?RESTARTTWI0?TWI
            CODE    044AH     0005H     UNIT         ?PR?INITINTERRUPT?MCU



OVERLAY MAP OF MODULE:   .\OBJ\5D_TWI0_M_P22P24_INT (MAIN)


SEGMENT                           BIT_GROUP 
  +--> CALLED SEGMENT          START    LENGTH
----------------------------------------------
?C_C51STARTUP                  -----    -----
  +--> ?PR?MAIN?MAIN

?PR?MAIN?MAIN                  -----    -----
  +--> ?PR?INITSYSTEM?MCU
  +--> ?CO?MAIN
  +--> ?PR?_TESTOUTSTR?FUNC
  +--> ?PR?TWI0PROC?TWI

?PR?INITSYSTEM?MCU             -----    -----
  +--> ?PR?INITPORT?MCU
  +--> ?PR?INITCLOCK?MCU
  +--> ?PR?INITTIMER?MCU
  +--> ?PR?INITUART0?MCU
  +--> ?PR?INITTWI0?MCU
  +--> ?PR?INITINTERRUPT?MCU

?PR?INITCLOCK?MCU              -----    -----
  +--> ?PR?_WRITEP?MCU

?PR?_WRITEP?MCU                0020H.1  0000H.1
  +--> ?PR?CHECKTRAPFLAG?MCU

?PR?_TESTOUTSTR?FUNC           -----    -----
  +--> ?PR?_TESTOUTBYTE?FUNC

?PR?TWI0PROC?TWI               -----    -----
  +--> ?PR?RESTARTTWI0?TWI
  +--> ?CO?TWI
  +--> ?PR?_TESTOUTSTR?FUNC
  +--> ?PR?_TESTOUTHEX?FUNC
BL51 BANKED LINKER/LOCATER V6.22                                                      11/20/2017  11:41:54  PAGE 3



?PR?_TESTOUTHEX?FUNC           -----    -----
  +--> ?PR?_TESTOUTBYTE?FUNC



SYMBOL TABLE OF MODULE:  .\OBJ\5D_TWI0_M_P22P24_INT (MAIN)

  VALUE           TYPE          NAME
  ----------------------------------

  -------         MODULE        MAIN
  C:0000H         SYMBOL        _ICE_DUMMY_
  D:0090H         PUBLIC        P1
  D:00A0H         PUBLIC        P2
  D:00C0H         PUBLIC        XICON
  D:00B0H         PUBLIC        P3
  D:00E8H         PUBLIC        P4
  D:00F8H         PUBLIC        P6
  D:00A8H         PUBLIC        IE
  D:00B8H         PUBLIC        IP0L
  D:0021H         PUBLIC        delayNmS
  D:00D8H         PUBLIC        CCON
  C:01D3H         PUBLIC        main
  D:0088H         PUBLIC        TCON
  B:00B0H.5       PUBLIC        P35
  D:0098H         PUBLIC        S0CON
  D:00C8H         PUBLIC        T2CON
  D:00E1H         PUBLIC        MG_WDTCR
  D:00D0H         PUBLIC        PSW
  -------         PROC          MAIN
  C:01D3H         LINE#         24
  C:01D3H         LINE#         25
  C:01D3H         LINE#         26
  C:01D6H         LINE#         27
  C:01DAH         LINE#         28
  C:01DDH         LINE#         30
  C:01DFH         LINE#         32
  C:01E8H         LINE#         34
  C:01EEH         LINE#         35
  C:01F4H         LINE#         36
  C:01F4H         LINE#         37
  C:01F5H         LINE#         38
  C:01F6H         LINE#         39
  C:01F7H         LINE#         40
  C:01F9H         LINE#         42
  C:01FDH         LINE#         43
  C:0200H         LINE#         45
  C:0202H         LINE#         47
  C:0205H         LINE#         48
  C:0208H         LINE#         49
  C:0208H         LINE#         50
  C:0208H         LINE#         51
  C:020BH         LINE#         52
  C:0211H         LINE#         53
  C:0211H         LINE#         54
  C:0216H         LINE#         55
BL51 BANKED LINKER/LOCATER V6.22                                                      11/20/2017  11:41:54  PAGE 4


  C:0218H         LINE#         56
  C:0218H         LINE#         58
  -------         ENDPROC       MAIN
  -------         ENDMOD        MAIN

  -------         MODULE        FUNC
  C:0000H         SYMBOL        _ICE_DUMMY_
  D:0090H         PUBLIC        P1
  D:00A0H         PUBLIC        P2
  D:00C0H         PUBLIC        XICON
  D:00B0H         PUBLIC        P3
  C:0307H         PUBLIC        _TestOutHex
  D:00E8H         PUBLIC        P4
  C:03F2H         PUBLIC        _NumberChk
  B:0020H.0       PUBLIC        bUartOutTxFlag
  D:00F8H         PUBLIC        P6
  D:00ACH         PUBLIC        SFRPI
  C:021AH         PUBLIC        INT_UART
  D:00A8H         PUBLIC        IE
  D:00B8H         PUBLIC        IP0L
  C:000EH         PUBLIC        _TestOutStr
  D:00D8H         PUBLIC        CCON
  D:0023H         PUBLIC        UartOutBufIn
  D:0024H         PUBLIC        UartOutBufOut
  D:0088H         PUBLIC        TCON
  C:02D4H         PUBLIC        _TestOutOCT
  B:00A8H.4       PUBLIC        ES0
  B:0098H.0       PUBLIC        RI0
  B:0098H.1       PUBLIC        TI0
  C:0261H         PUBLIC        _Bufcmp
  D:0099H         PUBLIC        S0BUF
  D:0098H         PUBLIC        S0CON
  D:00C8H         PUBLIC        T2CON
  C:029EH         PUBLIC        _Bufcpy
  C:0026H         PUBLIC        _TestOutByte
  X:0000H         PUBLIC        UartOutBuf
  D:00D0H         PUBLIC        PSW
  -------         PROC          INT_UART
  C:021AH         LINE#         7
  C:0222H         LINE#         9
  C:0224H         LINE#         10
  C:0227H         LINE#         11
  C:022AH         LINE#         12
  C:022AH         LINE#         13
  C:022CH         LINE#         14
  C:022CH         LINE#         15
  C:022FH         LINE#         16
  C:022FH         LINE#         17
  C:0231H         LINE#         18
  C:0236H         LINE#         19
  C:0236H         LINE#         20
  C:0238H         LINE#         21
  C:023AH         LINE#         23
  C:023AH         LINE#         24
  C:0248H         LINE#         25
  C:024AH         LINE#         26
  C:024CH         LINE#         27
BL51 BANKED LINKER/LOCATER V6.22                                                      11/20/2017  11:41:54  PAGE 5


  C:0253H         LINE#         28
  C:0253H         LINE#         29
  C:0256H         LINE#         30
  C:0256H         LINE#         31
  C:0256H         LINE#         32
  C:0256H         LINE#         33
  C:0258H         LINE#         34
  -------         ENDPROC       INT_UART
  -------         PROC          _TESTOUTBYTE
  D:0007H         SYMBOL        ToSend
  -------         DO            
  D:0006H         SYMBOL        i
  -------         ENDDO         
  C:0026H         LINE#         42
  C:0026H         LINE#         43
  C:0026H         LINE#         46
  C:0029H         LINE#         47
  C:0029H         LINE#         48
  C:002CH         LINE#         49
  C:002EH         LINE#         50
  C:003BH         LINE#         51
  C:003DH         LINE#         52
  C:003FH         LINE#         53
  C:0040H         LINE#         55
  C:0040H         LINE#         56
  C:0042H         LINE#         57
  C:004EH         LINE#         58
  C:004FH         LINE#         59
  C:0055H         LINE#         60
  C:0055H         LINE#         61
  C:0057H         LINE#         62
  C:0057H         LINE#         63
  C:005CH         LINE#         64
  C:005CH         LINE#         65
  C:005CH         LINE#         66
  C:005EH         LINE#         67
  C:0060H         LINE#         68
  C:0062H         LINE#         69
  C:0062H         LINE#         71
  -------         ENDPROC       _TESTOUTBYTE
  -------         PROC          _TESTOUTSTR
  D:0001H         SYMBOL        pStr
  C:000EH         LINE#         90
  C:000EH         LINE#         91
  C:000EH         LINE#         92
  C:0014H         LINE#         93
  C:0014H         LINE#         94
  C:0017H         LINE#         95
  C:001EH         LINE#         96
  C:0020H         LINE#         97
  -------         ENDPROC       _TESTOUTSTR
  -------         PROC          _TESTOUTOCT
  D:0005H         SYMBOL        ToSend
  -------         DO            
  D:0004H         SYMBOL        x
  -------         ENDDO         
  C:02D4H         LINE#         110
BL51 BANKED LINKER/LOCATER V6.22                                                      11/20/2017  11:41:54  PAGE 6


  C:02D6H         LINE#         111
  C:02D6H         LINE#         113
  C:02DCH         LINE#         114
  C:02E3H         LINE#         115
  C:02E6H         LINE#         116
  C:02E6H         LINE#         117
  C:02ECH         LINE#         118
  C:02ECH         LINE#         119
  C:02F2H         LINE#         120
  C:02F9H         LINE#         121
  C:0300H         LINE#         122
  -------         ENDPROC       _TESTOUTOCT
  -------         PROC          _TESTOUTHEX
  D:0005H         SYMBOL        ToSend
  -------         DO            
  D:0004H         SYMBOL        x
  -------         ENDDO         
  C:0307H         LINE#         141
  C:0309H         LINE#         142
  C:0309H         LINE#         144
  C:030EH         LINE#         145
  C:0314H         LINE#         146
  C:0314H         LINE#         147
  C:0316H         LINE#         148
  C:0318H         LINE#         150
  C:0318H         LINE#         151
  C:031EH         LINE#         152
  C:031EH         LINE#         153
  C:0322H         LINE#         154
  C:0328H         LINE#         155
  C:0328H         LINE#         156
  C:032AH         LINE#         157
  C:032CH         LINE#         159
  C:032CH         LINE#         160
  C:0332H         LINE#         161
  C:0332H         LINE#         162
  -------         ENDPROC       _TESTOUTHEX
  -------         PROC          _NUMBERCHK
  D:0007H         SYMBOL        uSou
  D:0005H         SYMBOL        uMin
  D:0003H         SYMBOL        uMax
  C:03F2H         LINE#         175
  C:03F2H         LINE#         176
  C:03F2H         LINE#         177
  C:03FAH         LINE#         178
  C:0402H         LINE#         179
  C:0404H         LINE#         180
  -------         ENDPROC       _NUMBERCHK
  -------         PROC          _BUFCMP
  D:0011H         SYMBOL        buf1
  D:0014H         SYMBOL        buf2
  D:0017H         SYMBOL        len
  -------         DO            
  D:0007H         SYMBOL        i
  -------         ENDDO         
  C:0261H         LINE#         192
  C:0267H         LINE#         193
BL51 BANKED LINKER/LOCATER V6.22                                                      11/20/2017  11:41:54  PAGE 7


  C:0267H         LINE#         195
  C:026FH         LINE#         196
  C:026FH         LINE#         197
  C:0298H         LINE#         198
  C:029BH         LINE#         199
  C:029DH         LINE#         200
  -------         ENDPROC       _BUFCMP
  -------         PROC          _BUFCPY
  D:0018H         SYMBOL        buf1
  D:001BH         SYMBOL        buf2
  D:001EH         SYMBOL        len
  -------         DO            
  D:0007H         SYMBOL        i
  -------         ENDDO         
  C:029EH         LINE#         211
  C:02A4H         LINE#         212
  C:02A4H         LINE#         214
  C:02ACH         LINE#         215
  C:02ACH         LINE#         216
  C:02D0H         LINE#         217
  C:02D3H         LINE#         218
  -------         ENDPROC       _BUFCPY
  -------         ENDMOD        FUNC

  -------         MODULE        MCU
  C:0000H         SYMBOL        _ICE_DUMMY_
  D:0095H         PUBLIC        P2M0
  D:0092H         PUBLIC        P2M1
  D:0090H         PUBLIC        P1
  D:00A0H         PUBLIC        P2
  D:00E7H         PUBLIC        ISPCR
  D:00C0H         PUBLIC        XICON
  D:00B0H         PUBLIC        P3
  D:00E8H         PUBLIC        P4
  C:03DCH         PUBLIC        InitClock
  D:00F8H         PUBLIC        P6
  B:00A8H.7       PUBLIC        EA
  D:00A8H         PUBLIC        IE
  I:0025H         PUBLIC        TrapFlag
  D:00B8H         PUBLIC        IP0L
  D:0093H         PUBLIC        T2MOD1
  C:0414H         PUBLIC        InitTimer
  C:035DH         PUBLIC        InitSystem
  D:00C7H         PUBLIC        CKCON0
  D:00BFH         PUBLIC        CKCON1
  D:00D8H         PUBLIC        CCON
  B:00C8H.5       PUBLIC        RCLK_TF2L
  D:00E6H         PUBLIC        SCMD
  D:00E3H         PUBLIC        IFADRH
  D:00E5H         PUBLIC        IFMT
  D:00E4H         PUBLIC        IFADRL
  D:0089H         PUBLIC        TMOD
  D:0088H         PUBLIC        TCON
  C:0436H         PUBLIC        InitTWI0
  C:0405H         PUBLIC        InitPort
  B:00A8H.4       PUBLIC        ES0
  B:00A8H.1       PUBLIC        ET0
BL51 BANKED LINKER/LOCATER V6.22                                                      11/20/2017  11:41:54  PAGE 8


  D:008CH         PUBLIC        TH0
  D:008DH         PUBLIC        TH1
  C:0384H         PUBLIC        INT_T0
  D:008AH         PUBLIC        TL0
  D:00E2H         PUBLIC        IFD
  B:0088H.4       PUBLIC        TR0
  B:0088H.6       PUBLIC        TR1
  C:0333H         PUBLIC        _WriteP
  D:0087H         PUBLIC        PCON0
  D:0098H         PUBLIC        S0CON
  C:03C6H         PUBLIC        InitUart0
  D:00C8H         PUBLIC        T2CON
  C:044AH         PUBLIC        InitInterrupt
  B:00C8H.4       PUBLIC        TCLK_TL2IE
  D:00A3H         PUBLIC        AUXR2
  D:00A4H         PUBLIC        AUXR3
  C:03A9H         PUBLIC        CheckTrapFlag
  D:00D0H         PUBLIC        PSW
  D:00D4H         PUBLIC        SICON
  -------         PROC          INT_T0
  C:0384H         LINE#         8
  C:0386H         LINE#         10
  C:0389H         LINE#         11
  C:038CH         LINE#         13
  C:039AH         LINE#         14
  C:03A0H         LINE#         15
  C:03A6H         LINE#         17
  -------         ENDPROC       INT_T0
  -------         PROC          INITINTERRUPT
  C:044AH         LINE#         26
  C:044AH         LINE#         27
  C:044AH         LINE#         28
  C:044CH         LINE#         29
  C:044EH         LINE#         31
  -------         ENDPROC       INITINTERRUPT
  -------         PROC          INITTWI0
  C:0436H         LINE#         39
  C:0436H         LINE#         40
  C:0436H         LINE#         41
  C:0439H         LINE#         42
  C:043AH         LINE#         43
  C:043BH         LINE#         44
  C:043CH         LINE#         45
  C:043FH         LINE#         48
  -------         ENDPROC       INITTWI0
  -------         PROC          INITTIMER
  C:0414H         LINE#         57
  C:0414H         LINE#         58
  C:0414H         LINE#         60
  C:0417H         LINE#         62
  C:041AH         LINE#         63
  C:041DH         LINE#         64
  C:041FH         LINE#         67
  -------         ENDPROC       INITTIMER
  -------         PROC          INITPORT
  C:0405H         LINE#         75
  C:0405H         LINE#         76
BL51 BANKED LINKER/LOCATER V6.22                                                      11/20/2017  11:41:54  PAGE 9


  C:0405H         LINE#         79
  C:040DH         LINE#         81
  C:0410H         LINE#         82
  C:0413H         LINE#         85
  -------         ENDPROC       INITPORT
  -------         PROC          INITUART0
  C:03C6H         LINE#         93
  C:03C6H         LINE#         94
  C:03C6H         LINE#         97
  C:03C9H         LINE#         99
  C:03CCH         LINE#         101
  C:03CFH         LINE#         102
  C:03D1H         LINE#         103
  C:03D3H         LINE#         106
  C:03D6H         LINE#         107
  C:03D9H         LINE#         109
  C:03DBH         LINE#         112
  -------         ENDPROC       INITUART0
  -------         PROC          INITCLOCK
  C:03DCH         LINE#         120
  C:03DCH         LINE#         121
  C:03DCH         LINE#         122
  C:03E0H         LINE#         124
  C:03E3H         LINE#         125
  C:03EAH         LINE#         126
  C:03EEH         LINE#         128
  C:03F1H         LINE#         130
  -------         ENDPROC       INITCLOCK
  -------         PROC          INITSYSTEM
  C:035DH         LINE#         139
  C:035DH         LINE#         140
  C:035DH         LINE#         142
  C:0361H         LINE#         143
  C:0364H         LINE#         145
  C:0367H         LINE#         146
  C:036AH         LINE#         147
  C:036EH         LINE#         148
  C:0371H         LINE#         149
  C:0374H         LINE#         150
  C:0377H         LINE#         151
  C:037AH         LINE#         153
  C:037DH         LINE#         154
  C:037FH         LINE#         155
  C:0381H         LINE#         157
  C:0383H         LINE#         158
  -------         ENDPROC       INITSYSTEM
  -------         PROC          _WRITEP
  D:0007H         SYMBOL        PsfrAddr
  D:0005H         SYMBOL        PsfrData
  -------         DO            
  B:0020H.1       SYMBOL        bEA
  -------         ENDDO         
  C:0333H         LINE#         188
  C:0333H         LINE#         189
  C:0333H         LINE#         190
  C:0337H         LINE#         191
  C:0339H         LINE#         192
BL51 BANKED LINKER/LOCATER V6.22                                                      11/20/2017  11:41:54  PAGE 10


  C:033CH         LINE#         193
  C:033EH         LINE#         194
  C:0340H         LINE#         195
  C:0343H         LINE#         196
  C:0346H         LINE#         197
  C:0349H         LINE#         198
  C:034CH         LINE#         199
  C:034FH         LINE#         200
  C:0352H         LINE#         201
  C:0353H         LINE#         202
  C:0356H         LINE#         203
  C:0358H         LINE#         204
  C:035CH         LINE#         205
  -------         ENDPROC       _WRITEP
  -------         PROC          CHECKTRAPFLAG
  C:03A9H         LINE#         213
  C:03A9H         LINE#         214
  C:03A9H         LINE#         215
  C:03BFH         LINE#         216
  C:03BFH         LINE#         218
  C:03C2H         LINE#         219
  C:03C5H         LINE#         220
  C:03C5H         LINE#         221
  -------         ENDPROC       CHECKTRAPFLAG
  -------         ENDMOD        MCU

  -------         MODULE        TWI
  C:0000H         SYMBOL        _ICE_DUMMY_
  D:0090H         PUBLIC        P1
  D:00A0H         PUBLIC        P2
  D:00C0H         PUBLIC        XICON
  D:00B0H         PUBLIC        P3
  D:00E8H         PUBLIC        P4
  D:00ADH         PUBLIC        EIE1
  D:00F8H         PUBLIC        P6
  D:00D3H         PUBLIC        SISTA
  D:00A8H         PUBLIC        IE
  D:0008H         PUBLIC        TWI0Runtime
  D:00B8H         PUBLIC        IP0L
  D:0009H         PUBLIC        SlaveDataLen
  D:000AH         PUBLIC        SlaveRegAddr
  D:000BH         PUBLIC        TWI0Ovtime
  D:000CH         PUBLIC        SlaveDataCnt
  D:00D8H         PUBLIC        CCON
  D:000DH         PUBLIC        TWI0Status
  D:0088H         PUBLIC        TCON
  B:00B0H.3       PUBLIC        P33
  C:0108H         PUBLIC        TWI0Proc
  D:000EH         PUBLIC        SlaveAddress
  D:000FH         PUBLIC        TWI0FailCnt
  D:0098H         PUBLIC        S0CON
  D:00C8H         PUBLIC        T2CON
  C:0440H         PUBLIC        ReStartTWI0
  C:0066H         PUBLIC        TWI0_ISR
  D:00D2H         PUBLIC        SIDAT
  D:0010H         PUBLIC        SlaveData
  D:00D0H         PUBLIC        PSW
BL51 BANKED LINKER/LOCATER V6.22                                                      11/20/2017  11:41:54  PAGE 11


  D:00D4H         PUBLIC        SICON
  -------         PROC          TWI0_ISR
  C:0066H         LINE#         7
  C:0075H         LINE#         9
  C:00A0H         LINE#         10
  C:00A0H         LINE#         11
  C:00A0H         LINE#         12
  C:00A3H         LINE#         13
  C:00A6H         LINE#         14
  C:00A8H         LINE#         15
  C:00A8H         LINE#         18
  C:00A8H         LINE#         19
  C:00ABH         LINE#         20
  C:00ADH         LINE#         21
  C:00ADH         LINE#         22
  C:00B0H         LINE#         23
  C:00B2H         LINE#         24
  C:00B2H         LINE#         27
  C:00B2H         LINE#         28
  C:00B5H         LINE#         29
  C:00BBH         LINE#         30
  C:00BDH         LINE#         32
  C:00BDH         LINE#         33
  C:00C0H         LINE#         34
  C:00C7H         LINE#         35
  C:00C7H         LINE#         36
  C:00C7H         LINE#         37
  C:00C9H         LINE#         43
  C:00C9H         LINE#         44
  C:00CCH         LINE#         45
  C:00CEH         LINE#         46
  C:00D8H         LINE#         47
  C:00D8H         LINE#         48
  C:00DBH         LINE#         49
  C:00DDH         LINE#         51
  C:00DDH         LINE#         52
  C:00E0H         LINE#         53
  C:00E0H         LINE#         54
  C:00E2H         LINE#         56
  C:00E2H         LINE#         57
  C:00E5H         LINE#         58
  C:00E8H         LINE#         59
  C:00EBH         LINE#         60
  C:00EDH         LINE#         61
  C:00EDH         LINE#         64
  C:00EDH         LINE#         65
  C:00EDH         LINE#         66
  C:00EDH         LINE#         67
  C:00F0H         LINE#         69
  C:00F0H         LINE#         70
  C:00F0H         LINE#         71
  C:00F5H         LINE#         72
  C:00F5H         LINE#         73
  C:00F8H         LINE#         74
  C:00F8H         LINE#         75
  C:00FBH         LINE#         77
  -------         ENDPROC       TWI0_ISR
BL51 BANKED LINKER/LOCATER V6.22                                                      11/20/2017  11:41:54  PAGE 12


  -------         PROC          RESTARTTWI0
  C:0440H         LINE#         85
  C:0440H         LINE#         86
  C:0440H         LINE#         87
  C:0443H         LINE#         88
  C:0444H         LINE#         89
  C:0445H         LINE#         90
  C:0446H         LINE#         91
  C:0449H         LINE#         92
  -------         ENDPROC       RESTARTTWI0
  -------         PROC          TWI0PROC
  C:0108H         LINE#         94
  C:0108H         LINE#         95
  C:0108H         LINE#         96
  C:0117H         LINE#         97
  C:0117H         LINE#         98
  C:0117H         LINE#         99
  C:011BH         LINE#         100
  C:011BH         LINE#         101
  C:011DH         LINE#         102
  C:0120H         LINE#         103
  C:0123H         LINE#         104
  C:0126H         LINE#         105
  C:0129H         LINE#         106
  C:012BH         LINE#         107
  C:012EH         LINE#         108
  C:0130H         LINE#         109
  C:0139H         LINE#         110
  C:013EH         LINE#         111
  C:013EH         LINE#         112
  C:013EH         LINE#         113
  C:013EH         LINE#         114
  C:013EH         LINE#         115
  C:013EH         LINE#         116
  C:0140H         LINE#         117
  C:0140H         LINE#         118
  C:0144H         LINE#         119
  C:0144H         LINE#         120
  C:0146H         LINE#         121
  C:0149H         LINE#         122
  C:014CH         LINE#         123
  C:014FH         LINE#         124
  C:0151H         LINE#         125
  C:0151H         LINE#         126
  C:0152H         LINE#         127
  C:0152H         LINE#         128
  C:0157H         LINE#         129
  C:015AH         LINE#         130
  C:015AH         LINE#         131
  C:015AH         LINE#         132
  C:015AH         LINE#         133
  C:015CH         LINE#         134
  C:015CH         LINE#         135
  C:015EH         LINE#         136
  C:0165H         LINE#         137
  C:0165H         LINE#         138
  C:0168H         LINE#         139
BL51 BANKED LINKER/LOCATER V6.22                                                      11/20/2017  11:41:54  PAGE 13


  C:016BH         LINE#         140
  C:016EH         LINE#         141
  C:0171H         LINE#         142
  C:0174H         LINE#         143
  C:0175H         LINE#         145
  C:0175H         LINE#         146
  C:0178H         LINE#         147
  C:017BH         LINE#         148
  C:017DH         LINE#         149
  C:017DH         LINE#         150
  C:017EH         LINE#         151
  C:017EH         LINE#         152
  C:0181H         LINE#         153
  C:0181H         LINE#         154
  C:0181H         LINE#         155
  -------         ENDPROC       TWI0PROC
  -------         ENDMOD        TWI

  -------         MODULE        ?C?CLDPTR
  C:0182H         PUBLIC        ?C?CLDPTR
  -------         ENDMOD        ?C?CLDPTR

  -------         MODULE        ?C?CSTPTR
  C:019BH         PUBLIC        ?C?CSTPTR
  -------         ENDMOD        ?C?CSTPTR

  -------         MODULE        ?C?CCASE
  C:01ADH         PUBLIC        ?C?CCASE
  -------         ENDMOD        ?C?CCASE

*** WARNING L16: UNCALLED SEGMENT, IGNORED FOR OVERLAY PROCESS
    SEGMENT: ?PR?_TESTOUTOCT?FUNC

*** WARNING L16: UNCALLED SEGMENT, IGNORED FOR OVERLAY PROCESS
    SEGMENT: ?PR?_NUMBERCHK?FUNC

*** WARNING L16: UNCALLED SEGMENT, IGNORED FOR OVERLAY PROCESS
    SEGMENT: ?PR?_BUFCMP?FUNC

*** WARNING L16: UNCALLED SEGMENT, IGNORED FOR OVERLAY PROCESS
    SEGMENT: ?PR?_BUFCPY?FUNC

Program Size: data=40.2 xdata=200 code=1100
LINK/LOCATE RUN COMPLETE.  4 WARNING(S),  0 ERROR(S)
